:10000000B6010E29A501A400B7172730A3001030B0
:1000100015200330A300E8301520A301643015201B
:10002000A3010A30152024082028A2002508A100D9
:100030002408A000D7202008031DB713B71B080011
:10004000303EA7000711871007108316071187108D
:100050000710F030860583122708B6184D283A306D
:10006000A1009830AA203330A60062201330A100EE
:100070008830AA2062206430A92062206430A92040
:100080002230A600622028304C200C304C20063054
:100090004C20B61427084D283614A600361C5B28C1
:1000A0008710033C031C602860200730A100D0307B
:1000B000AA20031408003614FE3C031909298714EA
:1000C000A60E361C36100715F030860526080F39A7
:1000D00086040711A60E361862283230A9200314B0
:1000E0000800A000A00DA00DA00D3830A0058130A3
:1000F00020049F000030A1003230AA201F151F19D4
:100100007F281E08A10083161E08092903178D00E9
:1001100083168C130C1483120C08092903178C0006
:1001200083168C130C1555308D00AA308D008C145D
:100130008C1898280C110929A301A200FF30A207EE
:10014000031CA307031C09290330A100E730AA20E0
:100150009E28A101FC3EA000A109031CB528FF3088
:100160000000A0070318B028A0076400A10FAF2863
:100170000800A2000230C728A301A2000330C7284C
:10018000A2000130C728A301A2000430C728A8009C
:1001900023082102031DCE28220820020430031860
:1001A0000130031902302805031DFF3009291030E2
:1001B000A600A501A401210DA40DA50D2208A402ED
:1001C0002308031C230FA5020318ED282208A40707
:1001D00023080318230FA5070310A00DA10DA60BDC
:1001E000DB28200809291030A800A101A001A70CD4
:1001F000A60C031C01292208A00723080318230FBB
:10020000A107A10CA00CA50CA40CA80BF72824088E
:100210000929831303138312640008008316FF3037
:10022000850082309F007030860081138701831221
:100230008501860187018A11AD29861783168613E9
:10024000FE308312212001302120483021206930E6
:100250002120203021204730212075302120793085
:10026000212073302120213021200330A300E830E9
:100270009D20FE302120C0302120503021207230BE
:1002800021206F30212064302120753021206330FF
:10029000212065302120643021202030212062304F
:1002A00021207930212020302120413021204F3061
:1002B000212052302120633021200730A300D0308C
:1002C0009D20080000307120BC002108BD000A30CC
:1002D0009C20080001307120C4002108C5000A30AC
:1002E0009C20080002307120C8002108C9000A3093
:1002F0009C20080003307120CC002108CD000A307A
:100300009C200800FE302120C0302120C93021204F
:10031000BA302120D83021205708A50056080320E4
:1003200030302120733021203A3021203F08A500B1
:100330003E080320DF3021202030212020302120E2
:100340002030212020302120203021202030212069
:1003500020302120203021200800851283168512AC
:100360008312DA01DB011D218613831686138312A3
:10037000851283168512053083128620DF00FE3039
:10038000212001302120B1302120B53021203A3008
:100390002120C0302120B2302120D4302120CB3088
:1003A0002120B0302120C430212020302120BA303B
:1003B0002120DD302120C4302120DB302120B0304D
:1003C0002120D7302120FE302120C0302120B7301D
:1003D0002120203021203A302120D3302120B0307C
:1003E0002120C0302120B0302120C4302120DE3037
:1003F0002120DA302120AF302120BB302120B03045
:1004000021200130A3002C309D2064008A11061F9A
:10041000102A8A1164008A11861EAE2C8A11052AC0
:1004200064309C2064008A11061F172A8A11FE304E
:10043000212001302120BE302120AF302120C330C7
:100440002120B2302120B5302120DD302120C430E0
:100450002120DE3021203D3021205F080220FE30A7
:100460002120C0302120B1302120B63021203A3067
:100470002120533021207430212020302120B7301A
:1004800021203A302120443021206E30212020309C
:100490002120B1302120B53021203A3021205530A3
:1004A000212070302120C8309C2064008A11061F52
:1004B000652A8A1164008A11861E702A8A116400D6
:1004C0008A11061E7B2A8A11552ADF0A64005030E1
:1004D0005F028A11031C6F2A8A115030DF00172A2D
:1004E000DF0364000B305F028A1103187A2A8A1135
:1004F0000A30DF00172A64309C206400061E7B2A25
:10050000031705308D0003135F088E20DA0A0319E4
:10051000DB0A5A08A0005B08A1000E30A3001030CF
:10052000C0208A11031D622C8A1162213C08A6009A
:100530003D08A7007D30A200A301F320B2002508EA
:10054000B3003208A0003308A100A2010130A300CB
:10055000D720BE002108BF006A214408A600450834
:10056000A7007D30A200A301F320B2002508B3004C
:100570003208A0003308A100A2010130A300D72057
:10058000C6002108C70072214808A6004908A70034
:100590007D30A200A301F320B2002508B300320889
:1005A000A0003308A100A2010130A300D720CA0097
:1005B0002108CB007A214C08A6004D08A7007D3009
:1005C000A200A301F320B2002508B3003208A00066
:1005D0003308A100A2010130A300D720CE002108DA
:1005E000CF003C084407B2003D080318013E450710
:1005F000B3004808B20749080318013EB3074C0886
:10060000B2074D080318013EB3073208A6003308AD
:10061000A7001930A200A301F320B2002508B300FF
:100620003208A0003308A100CD30A200A301D720DA
:10063000C2002108C300FE302120023021204130B9
:1006400021203F08A5003E0803203A3021204230F7
:1006500021204708A500460803203A3021204330D6
:1006600021204B08A5004A0803203A3021204430BD
:1006700021204F08A5004E08032020302120FE3005
:100680002120C03021204308A50042080320DF308C
:1006900021202D3021203E3021205F0802202030F3
:1006A00021206400061EB42905305F07B200B301A3
:1006B000B30D3E08A0003F08A1003308A300320894
:1006C000C0208A11031D142C8A1105305F07B20067
:1006D000B301B30D4608A0004708A1003308A300EA
:1006E0003208C0208A11031D142C8A1105305F07BF
:1006F000B200B301B30D4A08A0004B08A1003308B3
:10070000A3003208C0208A11031D142C8A11053061
:100710005F07B200B301B30D4E08A0004F08A1005F
:100720003308A3003208C0208A11031D142C8A113B
:100730004208A0004308A1005F08BC208A11031DE5
:100740003B2C8A1104305F07B200B301B30D3E08A1
:10075000A0003F08A1003308A3003208C4208A117A
:10076000031DF12B8A1104305F07B200B301B30DF2
:100770004608A0004708A1003308A3003208C4209F
:100780008A11031DF12B8A1104305F07B200B301F7
:10079000B30D4A08A0004B08A1003308A30032089B
:1007A000C4208A11031DF12B8A1104305F07B200A7
:1007B000B301B30D4E08A0004F08A1003308A300F9
:1007C0003208C4208A11031DF12B8A114208A000AF
:1007D0004308A1005F08C3208A11031DF12B8A1171
:1007E000862A85168316851283128617831686132A
:1007F000FE3083122120C73021202B3021204830A9
:100800002120653021206130212074302120693081
:1008100021206E302120673021202130212003301B
:10082000A300B9309D20862A851283168512831273
:10083000861383168613FE3083122120C7302120B1
:100840002130212031302120D8302120DD302120DD
:1008500020302120BA302120B3302120B530212092
:10086000DD3021200330A300B9309D208617831688
:1008700086138312862A85128316851283128613A5
:1008800083168613FE3083122120C73021202D309D
:100890002120CE302120B5302120DD302120C13073
:1008A0002120AD302120B3302120203021202030E4
:1008B00021200330A300B9309D20861783168613AC
:1008C0008312862A851283168512FE308312212018
:1008D0000130212031302120BC302120DE30212088
:1008E000B6302120DD302120B2302120BC30212043
:1008F000DE302120AE302120B3302120B93021203C
:10090000B2302120B6302120FE302120C0302120FD
:10091000B1302120DD302120BE302120DE302120E9
:10092000DD302120C9302120C0302120D2302120CB
:100930004F3021204630212046302120BC3021205C
:10094000CF302120BC302120C030212086138316D7
:10095000861383126400061EB429AA2C64309C20DE
:100960006400861EAE2C861383168613063083120F
:100970008620DE0007308620DD0008308620C0009B
:10098000C10109308620DC005D08A600A701A20194
:100990000130A300F320B2002508B3005E0832073F
:1009A000D60033080318013ED700FE302120013065
:1009B0002120C3302120B2302120BC302120B5308D
:1009C0002120DD302120C4302120DE3021203D30A7
:1009D00021204108A50040080320DF302120FE30FF
:1009E0002120C0302120B1302120B63021203A30E2
:1009F00021204E3021207830212020302120B73096
:100A000021203A302120443021206E302120203016
:100A10002120B1302120B53021203A30212055301D
:100A200021207030212096309C2064008A11061FFE
:100A3000252D8A1164008A11861E372D8A116400C3
:100A40008A11061E4C2D8A11152DC00A0319C10AE0
:100A50004008A0004108A100A3015A30C4208A1117
:100A6000031D362D8A115A30C000C101D52C01302A
:100A7000C0020030031C013EC1024008A000410832
:100A8000A100A3010A30C0208A11031D4B2D8A1139
:100A90000A30C000C101D52C64309C206400061EC1
:100AA0004C2DFE302120013021205430212069308E
:100AB00021206D30212065302120723021203D30F1
:100AC00021205708A500560803203030212073301C
:100AD00021206530212063302120FE302120C030CC
:100AE0002120B1302120B63021203A3021204E3053
:100AF00021207830212020302120B73021203A30A9
:100B00002120443021206E30212020302120B1309E
:100B10002120B53021203A3021205530212070305D
:100B2000212096309C2064008A11061FA32D8A1173
:100B300064008A11861EB72D8A1164008A11061E70
:100B4000CC2D8A11932DD60A0319D70A5608A00076
:100B50005708A100FD30A3002030C4208A11031DD6
:100B6000B62D8A112030D600FD30D700512D01302E
:100B7000D6020030031C013ED7025608A0005708D9
:100B8000A100A3010130C0208A11031DCB2D8A11C1
:100B90000130D600D701512D64309C206400061E20
:100BA000CC2DFE302120013021204C3021206F300F
:100BB00021207730212065302120723021204430DF
:100BC00021207530212074302120793021203D30C2
:100BD00021205C08022025302120FE302120C03059
:100BE0002120B1302120B63021203A3021204E3052
:100BF00021207830212020302120B73021203A30A8
:100C00002120443021206E30212020302120B1309D
:100C10002120B53021203A3021205530212070305C
:100C2000212096309C2064008A11061F232E8A11F1
:100C300064008A11861E2E2E8A1164008A11061EF7
:100C4000392E8A11132EDC0A640046305C028A11A8
:100C5000031C2D2E8A114630DC00D12DDC036400EC
:100C600003305C028A110318382E8A110230DC002E
:100C7000D12D5608DE005608A0005708A100A20199
:100C80000130A300D720DD00031706308D000313C9
:100C90005E088E20031707308D0003135D088E2039
:100CA000031708308D00031340088E200317093006
:100CB0008D0003135C088E20FE302120013021209E
:100CC000B6302120B2302120C3302120DD30212058
:100CD000BD302120B330212020302120B63021200A
:100CE000CD302120DD30212020302120C5302120B1
:100CF000D7302120BC302120203021203F3021203E
:100D0000FE302120C0302120B73021203A30212070
:100D10004E3021206F30212020302120B130212081
:100D2000B53021203A302120593021206530212052
:100D30007330212064008A11861EA52E8A1164005A
:100D40008A11061F3B2F8A119A2EFE302120013076
:100D50002120443021207530212074302120793029
:100D600021203D3021205C080220253021203A300E
:100D700021204330212075302120743021203D3046
:100D800021204108A50040080320DF3021208221D6
:100D90008617831686138312D401D5015408A00048
:100DA0005508A100B630A3006C30C0208A11031D85
:100DB000FE2E8A11851683168512031083125C0D90
:100DC000B200B301B30D3308A1003208AA20851286
:100DD0008316851283125C08643CB2000030031C49
:100DE000FF3EB3000310B20DB30D3308A10032086B
:100DF000AA20D40A0319D50A031DCE2E0030712073
:100E0000BC002108BD003C08A6003D08A7007D30BD
:100E1000A200A301F320B2002508B3003208A0000D
:100E20003308A100A2010130A300D720BE00210891
:100E3000BF000130D6020030031C013ED7028221E0
:100E40006400061EB4295608A0005708A100A3019B
:100E50000030B9208A15031D6A288A113E08A000B7
:100E60003F08A1004108A3004008BD208A15031DCA
:100E70009C288A11CC2EFE302120013021205C08D4
:100E8000022025302120743021206F3021200A30AB
:100E90005C07B200B301B30D3308A500320803208C
:100EA000253021203A302120433021207530212067
:100EB000743021203D3021204108A5004008032046
:100EC000DF30212082218617831686138312D201F8
:100ED000D3015208A0005308A100A3011430C02080
:100EE0008A11031DBC2F8A11D401D5015408A0001A
:100EF0005508A1000430A3007D30C0208A11031DD5
:100F0000B72F8A11851683168512031083125C0D84
:100F1000B200B301B30D5208B20753080318013EE3
:100F2000B3073308A1003208AA2085128316851260
:100F300083125208C83CB2005308031C013E003C17
:100F4000B30003105C0DB400B501B50D34083202D6
:100F5000B4003508031C013E3302B5003508A1007A
:100F60003408AA20D40A0319D50A031D762FD20A01
:100F70000319D30A031D692F861383168613831260
:100F80001330D200D3015208A0005308A100A301DE
:100F90000130C4208A15031D1E288A11D401D501F1
:100FA0005408A0005508A1000430A3007C30C020E4
:100FB0008A15031D16288A118516831685120310BB
:100FC00083125C0DB200B301B30D5208B20753088F
:100FD0000318013EB3073308A1003208AA20851286
:100FE0008316851283125208C83CB2005308031CB2
:100FF000013E003CB30003105C0DB400B501B50D1B
:1010000034083202B4003508031C013E3302B50037
:101010003508A10034088A158A11AA208A15D40A35
:101020000319D50A8A11031DD02F8A150130D20267
:10103000031CD3028A110318C32F8A1500308A11AA
:1010400071208A15BC002108BD003C08A6003D089F
:10105000A7007D30A200A3018A11F3208A15B200F7
:101060002508B3003208A0003308A100A201013016
:10107000A3008A11D7208A15BE002108BF000130C5
:10108000D6020030031C013ED7028A1182218A1544
:1010900064008A11061EB4298A155608A000570854
:1010A000A100A30100308A11B9208A158A15031DF9
:1010B0006A288A153E08A0003F08A1004108A30045
:1010C00040088A11BD208A158A15031D9C288A159F
:1010D0008A11632F85128316851283128613831655
:1010E0008613FE308A11831221208A1501308A115D
:1010F00021208A15C5308A1121208A15D7308A11FE
:1011000021208A15BC308A1121208A15B6308A1117
:1011100021208A15DD308A1121208A15D8308A11C4
:1011200021208A15AE308A1121208A15B3308A1108
:1011300021208A158A11AA2C861383168613FE3065
:101140008A11831221208A1501308A1121208A15E3
:10115000D3308A1121208A15B0308A1121208A15B6
:10116000C0308A1121208A15B0308A1121208A15B9
:10117000B5308A1121208A15DD308A1121208A1587
:10118000C4308A1121208A15DE308A1121208A1567
:10119000C1308A1121208A15AE308A1121208A158A
:1011A000B3308A1121208A15B6308A1121208A1580
:1011B00021308A1121208A158A11AA2C6300DE2889
:02400E00723D01
:0A420A0028001200000032000A0034
:00000001FF
